:1000000001308A007F2900002D308400831300080E
:10001000031917280230F800F701F70B0D28F80B29
:100020000C289730F700F70B1328800B0A280800DC
:1000300005110517071287120717071187100714F4
:100040008715851105158A110A126C2A0714871560
:10005000B6013608073C031C3828B41F31280715A1
:1000600032280711871487100310B40DB60A292807
:10007000B6013608073C031C4828B51F4128071560
:1000800042280711871487100310B50DB60A3928C6
:1000900008003208B4003308B50026200710071402
:1000A00008003208B4003308B500262087118715F0
:1000B0000800051105130712871607170711871087
:1000C00007148715851105150130AD000420123085
:1000D000B2008030B30049201430B2008030B30049
:1000E00051208A110A126C2A05110513071687126E
:1000F000071707118710071487158511051501309B
:10010000AD0004201230B2008030B300492014301A
:10011000B2008030B30051208A110A126C2A0511F6
:100120000513071287120713071187100714871585
:10013000851105150130AD0004201230B200B30165
:1001400049201430B200B30151208A110A126C2ADE
:1001500005110513071687160713071187100714D3
:100160008715851105150130AD0004201230B2004D
:10017000B30149201430B200B30151208A110A1290
:100180006C2AB301B201B40134080F3C031CEA2805
:100190009F1435109F1C35143518D22835109F1C1C
:1001A0003514CC289F18D2281E08FA0083161E0882
:1001B0008312B6001E08B7003608F8003708F900A9
:1001C0007908FA007808B20779080318790FB3079D
:1001D000B40AC428B30CB20CB30CB20CB30CB20CFE
:1001E000B30CB20C0F30B305220B242921083302C3
:1001F000031C0829031D00293208200203180829BE
:100200003308A1003208A000F8002108F90056299F
:1002100001303207F8003308FA000318FA0A7A08A6
:100220002102031C2329031D192920087802031821
:1002300023293308A1003208A000A2012008F800F9
:100240002108F9005629522933082102031C3629B6
:10025000031D2E2920083202031836293308A10075
:100260003208A000F8002108F900562901302007C3
:10027000B5002108B6000318B60A36083302031C7D
:100280005229031D47293208350203185229330821
:10029000A1003208A0000130A2002008F8002108C7
:1002A000F90056292008F8002108F9007908AD0066
:1002B0007808AC0023082C02031D622924082D02B3
:1002C00003197C292D08A4002C08A3002C08AF00DA
:1002D000B3012D080339AE002E080438B0002E08F3
:1002E0000C38B1003008B2002F08B30049203108A3
:1002F000B2002F08B30051208A110A126E2A84011D
:1003000083131F308305713083168F000F0883120B
:10031000A101A0010130A2000330A400FF30A3001E
:10032000FF30A500831603170908C039890003139D
:100330001F129F1200300317880083128701880163
:100340008901FF3083160313950081138500860011
:1003500087008612831286128316061383120613F1
:1003600083168613831286130430AC00FA30AD0076
:100370000420AC0BB6290430AC00FA30AD000420E8
:10038000AC0BBD290430AC00FA30AD000420AC0B3E
:10039000C4290430AC00FA30AD000420AC0BCB29EA
:1003A0000430AC00FA30AD000420AC0BD2291F138E
:1003B0009F1783169F1783121F14831603170908AC
:1003C000C039890003131F129F12013003178800E0
:1003D0000030F800831203131F08C33978049F000C
:1003E000A5132508831687008510051105128512AF
:1003F000851305118312051183168511831285114A
:10040000251025088316870083120714A5112508D7
:100410008316870083128715A51025088316870089
:100420008312871425112508831687008312071568
:1004300083160513831205172512250883168700D6
:1004400083120712A51225088316870083128712CC
:100450002513250883168700831207170515013019
:10046000AD0004200530A600AB01AA012B08A900AD
:100470002A08A800A70106183F2A0130A7008618FD
:10048000432A0230A7000619472A0330A70086191D
:100490004B2A0430A7002708260203196C2A2708D4
:1004A000A60026080319612A013A0319632A033AB0
:1004B0000319652A013A0319672A073A0319692AB9
:1004C0006B2A18286C2A59286C2A74286C2A8F28C1
:1004D0006C2AA8286C2A6C2A8616C128861229083C
:1004E000023C03187C2AFF3A031D7A2A2808E83CBC
:1004F00003187C2A06177F2AA80A0319A90A2B08C1
:10050000083C03188C2AFF3A031D8A2A2A08C43C97
:1005100003188C2A86178F2AAA0A0319AB0A3A2ACB
:02052000630076
:04400E00842CFF3FC0
:00000001FF
